:100000000C944B000C9466000C9466000C946600F3
:100010000C9466000C9466000C9466000C946600C8
:100020000C9466000C9466000C9466000C946600B8
:100030000C9466000C9466000C9466000C946600A8
:100040000C9466000C9466000C9466000C94660098
:100050000C946600663D2078782E7878782E787833
:100060002047487A64662F64743D20202020207049
:10007000706D2F73004672657175656E6379636F7D
:10008000756E74657256657220332E3020202044C0
:100090004C354E45470011241FBECFE5D4E0DEBFEE
:1000A000CDBF10E0A0E6B0E0E6E3F3E102C00590CA
:1000B0000D92A636B107D9F710E0A6E6B0E001C070
:1000C0001D92AB3CB107E1F70C94D1030C940000F6
:1000D000AC0183E083BF20E030E02417350768F4EB
:1000E00096EC92BF88B7816088BF08B600FEFDCF4E
:1000F0002F5F3F4F24173507A0F30895CF93DF9369
:10010000AB01BC012FE030E0C6EAD0E0FE0134973D
:1001100080819181A281B38188839983AA83BB83E3
:1001200021503040EF011216130684F340936A0009
:1001300050936B0060936C0070936D0020E030E092
:1001400040E050E0EAE6F0E081919191A191B19117
:10015000280F391F4A1F5B1F80E0E63AF807A1F31A
:100160009CF384E055954795379527958A95D1F767
:1001700020936600309367004093680050936900B5
:10018000DF91CF910895809160008F5F8093600030
:10019000853010F01092600080916000882361F437
:1001A00081E38093BB0080E28093BC008093BD001C
:1001B0008093BE008DE43DC0813051F486E380938E
:1001C000BB0084E38093BC0080E28093BD000CC040
:1001D0008230A9F481E38093BB0082E38093BC006A
:1001E00088E38093BD0080E28093BE0087E4809323
:1001F000B6008EE28093AD008093B10021C08330C1
:1002000059F486E38093BB0084E38093BC0080E3D1
:100210008093BD0080E20AC0843091F481E3809332
:10022000BB0080E38093BC008093BD008093BE0040
:1002300087E48093B6008EE28093AE008093B20094
:1002400088EC90E00E946800089598B39F7098BB76
:10025000982F907F88B3892B88BB959A959881E0D9
:1002600090E00E94680008951F93CF93DF939698C3
:1002700080E80E94250180E00E9425018FE090E047
:100280000E946800969ACAEAD0E01FE08881807FC9
:100290000E94250189918295807F0E94250111503D
:1002A00017FFF4CF969880EC0E94250180E00E9411
:1002B00025018FE090E00E946800969ACAEBD0E09A
:1002C0001FE08881807F0E94250189918295807F2F
:1002D0000E942501115017FFF4CFDF91CF911F919C
:1002E0000895CF938FE090E00E94680082B38F79E9
:1002F00082BBC2E080E30E94250185E090E00E947D
:100300006800C150C7FFF6CF80E20E94250185E05A
:1003100090E00E94680080E20E94250180E80E942F
:10032000250185E090E00E94680080E00E942501A0
:1003300080E10E94250185E090E00E94680080E055
:100340000E94250180E60E94250185E090E00E9440
:10035000680080E00E94250180EC0E94250185E074
:1003600090E00E946800CF910895EF92FF920F9362
:100370001F93CF93DF93CDB7DEB764970FB6F89492
:10038000DEBF0FBECDBF7B018C019F938F937F9308
:100390006F9381E690E09F938F93CE0101969F9398
:1003A0008F930E94B9048DB79EB708960FB6F89444
:1003B0009EBF0FBE8DBF90EAE91696E8F90691E060
:1003C000090790E01907E4F48C818093C0008D81C7
:1003D0008093C1008E818093C2008F818093C3007F
:1003E00088858093C40080E78093C5008093C60011
:1003F0008DE68093C7008FE28093C80083E71AC020
:100400009FE69093C00086E78093C10085E68093C5
:10041000C20082E78093C30086E68093C4008CE626
:100420008093C5009093C60087E78093C70080E261
:100430008093C8008093C90064960FB6F894DEBF1D
:100440000FBECDBFDF91CF911F910F91FF90EF9025
:100450000895EF92FF920F931F93CF93DF93CDB741
:10046000DEB764970FB6F894DEBF0FBECDBF7B0139
:100470008C0180916000882309F03FC0C801B7015A
:1004800024E630E040E050E00E945A097B018C01F4
:1004900047E016950795F794E7944A95D1F71F938F
:1004A0000F93FF92EF9281E690E09F938F93CE019E
:1004B00001969F938F930E94B90489818093AC0029
:1004C0008A818093AD008B818093AE008C81809374
:1004D000B0008D818093B1008E818093B2008F81B6
:1004E0008093B40088858093B5008DB79EB7089639
:1004F0000FB6F8949EBF0FBE8DBF80916000813013
:1005000079F516950795F794E7941F930F93FF924B
:10051000EF9281E690E09F938F93CE0101969F9397
:100520008F930E94B9048A818093AC008B81809361
:10053000AE008C818093AF008D818093B0008E815E
:100540008093B2008F818093B30088858093B4003C
:100550008DB79EB708960FB6F8949EBF0FBE8DBF9D
:1005600080916000823059F51F930F93FF92EF92B4
:1005700081E690E09F938F93CE0101969F938F9396
:100580000E94B9048A818093AC008B818093AE0075
:100590008C818093AF008D818093B0008E81809399
:1005A000B2008F818093B30088858093B4008DB7AB
:1005B0009EB708960FB6F8949EBF0FBE8DBF809170
:1005C0006000833091F516950795F794E7941F9393
:1005D0000F93FF92EF9281E690E09F938F93CE016D
:1005E00001969F938F930E94B90489818093AB00F9
:1005F0008A818093AC008B818093AD008C81809345
:10060000AF008D818093B0008E818093B1008F8187
:100610008093B30088858093B4008DB79EB7089609
:100620000FB6F8949EBF0FBE8DBF809160008430DE
:1006300009F03FC0C801B70124E630E040E050E0D7
:100640000E945A097B018C0197E016950795F79453
:10065000E7949A95D1F71F930F93FF92EF9281E65B
:1006600090E09F938F93CE0101969F938F930E946A
:10067000B90489818093AC008A818093AD008B811D
:100680008093AE008C818093B0008D818093B10007
:100690008E818093B2008F818093B400888580938F
:1006A000B5008DB79EB708960FB6F8949EBF0FBEE3
:1006B0008DBF0E94340164960FB6F894DEBF0FBE62
:1006C000CDBFDF91CF911F910F91FF90EF900895D3
:1006D000805D8A3308F0895F99270895EF92FF9231
:1006E0000F931F937B018C01DC01CB012CE1B695AC
:1006F000A795979587952A95D1F78F700E946803E3
:100700008093C200812F9927AA27BB278F700E9450
:1007100068038093C300D801C701F4E1B695A7959B
:1007200097958795FA95D1F78F700E94680380930B
:10073000C400C801AA27BB278F700E94680380935A
:10074000C500D801C7017CE0B695A7959795879518
:100750007A95D1F78F700E9468038093C600BB27FB
:10076000A12F902F8F2D8F700E9468038093C70058
:10077000D801C70154E0B695A795979587955A95E6
:10078000D1F78F700E9468038093C8008E2D8F7000
:100790000E9468038093C9001F910F91FF90EF9012
:1007A0000895CFE5D4E0DEBFCDBFEE24FF2487015E
:1007B00086E08EBD8A9A80EF87BB81B3806681BB5D
:1007C000939A979A0E94710165E770E08AEA90E037
:1007D0000E94B2040E94340180ED97E00E946800FC
:1007E00064E570E08AEA90E00E94B2040E9434015D
:1007F000849BFECF8499FECF81E090E00E94680048
:1008000026B322702295220F220F207C83B38F778C
:10081000282B8CB5482F55278DB599275C01CC2402
:10082000DD246501BB24AA24942F8827AA27BB278F
:10083000A80EB91ECA1EDB1EA20EB11CC11CD11C03
:10084000879904C0C601B5010E946E03C601B501B7
:100850000E942902C801B7016A197B098C099D0908
:10086000A114B104C104D10429F431E0A32EB12CA8
:10087000C12CD12C0E9498087B018C01C601B501C6
:100880000E949808DC01CB019C01AD01C801B701B1
:100890000E943508DC01CB0120E034E244E759E452
:1008A000BC01CD010E94120920E030E04AE754E487
:1008B0000E941209DC01CB0120E030E040E05CE363
:1008C000BC01CD010E9412097B018C0120E030E5C2
:1008D00043EC57E40E94A508181654F40F2EF0E0DC
:1008E000EF2EF0E5FF2EF3EC0F2FF7E41F2FF02D86
:1008F00020E030E040E050E0C801B7010E94A508C8
:1009000088234CF020E030E040E05FE3C801B7010D
:100910000E94F30708C020E030E040E05FE3C80138
:10092000B7010E94F207DC01CB01BC01CD010E949E
:100930007B080E947E008091660090916700A091E4
:100940006800B0916900BC01CD010E94B501929A86
:1009500092981DBC1CBC839902C00E94C3008601F2
:10096000750146CFFB01DC0105900D920020E1F7F7
:1009700008950F931F93CF93DF93CDB7DEB72E97D4
:100980000FB6F894DEBF0FBECDBF0D891E892F892B
:10099000388D86E08C831A8309838FEF9FE79E83CF
:1009A0008D83AE01475E5F4FB901CE0101960E9473
:1009B000E904EF81F885E00FF11F10822E960FB643
:1009C000F894DEBF0FBECDBFDF91CF911F910F9185
:1009D00008952F923F924F925F926F927F928F92E3
:1009E0009F92AF92BF92CF92DF92EF92FF920F93BE
:1009F0001F93CF93DF93CDB7DEB762970FB6F8940E
:100A0000DEBF0FBECDBFEE24FF2487011C017E8711
:100A10006D872A01CC24DD24FC01D782C682838124
:100A200081FD68C28FEF9FEF78C28D859E8501960C
:100A30009E878D87C0FE4BC28F8580538A30D0F44D
:100A40009F85903339F4662029F4C3FC03C0E0E0AD
:100A5000F1E08DC08AE0689E602C1124FF856F0E46
:100A600020ED620E67FE02C05FE7652EC3FC42C246
:100A7000762C40C2C3FE04C0662011F441E0642E0F
:100A8000EF858E2F992787FD9095883691058CF5F7
:100A9000853691050CF06EC08335910509F493C03D
:100AA00084359105CCF48B32910509F449C08C3220
:100AB00091054CF48032910509F446C083329105CA
:100AC00009F44AC0FEC18D32910509F440C08E324E
:100AD000910509F444C0F5C18336910509F450C06D
:100AE000843691050CF08AC08835910509F4BCC0A4
:100AF000E8C18037910509F4B1C08137910584F4CC
:100B00008C36910591F18D3691052CF4893691053D
:100B100009F474C0D6C18F36910509F49CC0D1C1C7
:100B20008537910509F4A2C08637910524F48337EF
:100B3000910571F1C6C18837910509F495C0C1C10D
:100B400080E190E0C82AD92AE0E2F0E010C080E815
:100B500090E0C82AD92ACEC1E0E4F0E008C088E0DD
:100B600090E0C82AD92A6624C5C1E4E0F0E0CE2A84
:100B7000DF2AC0C13FE3E32E7A94F3E6FF873CC14E
:100B8000F20182E090E0480E591EE0807A9434C170
:100B9000F20182E090E0480E591EA081B1817D01F2
:100BA000C3FE09C0862D992787FD9095BC01CD0114
:100BB0000E94BA071FC0FD0101900020E9F731979C
:100BC000EA1BE88B18C0F20182E090E0480E591E43
:100BD0000190F081E02D7F01C3FE09C0862D992789
:100BE00087FD9095BC01CF010E94AF0703C0CF01E4
:100BF0000E94A607888B9889791AFEC0C2FE0AC097
:100C0000F20184E090E0480E591E2081318142813A
:100C100053810CC0F20182E090E0480E591E8081A1
:100C200091819C01442737FD4095542F79018A0119
:100C300057FF0CC0E2E0F0E0CE2ADF2A10950095C5
:100C4000F094E094E11CF11C011D111D8FEB9FEF4E
:100C5000C822D92227C098E0988B08C0E0E4F0E0D1
:100C6000CE2ADF2AF8E7FF8720E1288BC2FE0AC0E0
:100C7000F20184E090E0480E591E208131814281CA
:100C800053810AC0F20182E090E0480E591E808133
:100C900091819C014427552779018A01EFECFFEFF0
:100CA000CE22DF22CE0101969A8B898B9889892EDC
:100CB0009924AA24BB24C801B701A50194010E946C
:100CC0007909DC01CB01E989FA8980838A3024F033
:100CD000FF858F0F815201C0805DE989FA89819378
:100CE000FA8BE98BC801B701A50194010E9479092B
:100CF00079018A012115310541055105E1F6E9889F
:100D000081E090E08C0F9D1FE81AC60182739070FD
:100D1000892B09F07A94C6FE0DC0872D992787FD8F
:100D20009095E889E03121F42EEF722E780E02C002
:100D3000782E7A94C3FE0FC0262D332727FD3095D9
:100D40008E2D9927821793072CF087EF9FEFC822EB
:100D5000D92201C06E18C3FE02C0761801C07E18E9
:100D6000C60180789170892B51F4872D7A941816DA
:100D700034F4B10180E290E00E94C507F6CFC1FED5
:100D800004C0B1018DE290E00BC0C4FE04C0B1010B
:100D90008BE290E005C0C5FE05C0B10180E290E0A5
:100DA0000E94C507C6FE10C0B10180E390E00E941A
:100DB000C5079889903141F4B101EF858E2F9927AD
:100DC00087FD90950E94C507D0FE0AC0872D7A94B2
:100DD000181634F4B10180E390E00E94C507F6CF05
:100DE000C3FE0AC0862D6A94181634F4B10180E35C
:100DF00090E00E94C507F6CF90E8B92EBC2051F4D0
:100E0000872D7A94181634F4B10180E290E00E94A4
:100E1000C507F6CFFF85F33641F48E2DB101992732
:100E200087FD90950E94C50740C02F852337B1F4F8
:100E300088898150888B8F3FC1F1F70180810894A8
:100E4000E11CF11CB101992787FD90950E94C5070F
:100E500098899150988B9F3F81F727C0EF85E335A4
:100E600079F4F889F150F88BFF3FF9F0F70184919C
:100E7000B10199270E94C5070894E11CF11CF1CF2C
:100E80006E010894C11CD11C89899A898C159D0515
:100E900061F0E989FA898291FA8BE98BB10199278E
:100EA00087FD90950E94C507EFCFBB2069F0872D85
:100EB0007A9418164CF4B10180E290E00E94C507C4
:100EC000F6CFB1010E94C507CC24DD2413C09F8555
:100ED000953241F481E0C82ED12C6624762CEAE0CC
:100EE000E88B08C0B101FF858F2F992787FD90956A
:100EF0000E94C507F101838183FF04C0ED85FE8553
:100F0000F49103C0ED85FE85F081FF872F852223B4
:100F100009F08BCDF1018681978162960FB6F89426
:100F2000DEBF0FBECDBFDF91CF911F910F91FF901C
:100F3000EF90DF90CF90BF90AF909F908F907F9079
:100F40006F905F904F903F902F900895FC01059017
:100F50000020E9F7809590958E0F9F1F0895FC0162
:100F60000590615070400110D8F7809590958E0FD4
:100F70009F1F0895FC016150704001900110D8F747
:100F8000809590958E0F9F1F08950F931F93CF9379
:100F9000DF938C01EB018B81992781FF1CC082FFBD
:100FA0000DC02E813F818C819D812817390764F403
:100FB000E881F9810193F983E88306C0E885F98522
:100FC000802F0995892B39F48E819F8101969F830B
:100FD0008E83C80102C08FEF9FEFDF91CF911F91E9
:100FE0000F9108955058192EEFD001D0D2C0BA17E2
:100FF0006207730784079507B1F188F40EF4109423
:101000000B2EBA2FA02D062E622F202D072E732F08
:10101000302D082E842F402D092E952F502DFF277F
:101020005523B9F0591B49F0573E98F0469537952E
:101030002795A795F0405395C9F776F0BA0F621F30
:10104000731F841F30F4879577956795B795F040A7
:10105000939517FA0F2E0895BF1BBB27BA0B620B8F
:10106000730B840BF6CFDEF6DBC0AED001D091C09F
:10107000552359F0992369F09F575F57951B33F417
:1010800042F4903811F4915805C09BC091589F3F8D
:1010900009F4C6C0BB27112462177307840730F414
:1010A000660F771F881FBB1F915098F311D00F92C6
:1010B0000FD00F920DD0A0E82617370748071B0660
:1010C00009F0A048BA2F602D7F918F9100240895D8
:1010D000A0E80024621773078407B10528F0621B9B
:1010E000730B840BB1090A2A660F771F881FBB1F79
:1010F000A69581F7089597FB73D09F3738F0FEE9E6
:10110000F91B982F872F762F6B2F05C086C09695D9
:10111000879577956795F150D0F73EF49095809537
:10112000709561957F4F8F4F9F4F0895E89403C04E
:1011300097FB0EF4F3DFB62F672F782F892F9EE9E8
:10114000002427C00ED05EF004C00BD026F001C0F2
:1011500008D019F020F48FEF089580E0089581E021
:10116000089597FB092E052600F8689430D0E8947E
:1011700007FC07C0621773078407950721F008F47E
:1011800000940794989408959A95BB0F661F771F53
:10119000881F11249923A1F08823B2F79F3F59F0AB
:1011A000BB0F48F421F4002011F460FF04C06F5F0E
:1011B0007F4F8F4F9F4F881F9795879597F9089579
:1011C0002CC09FEF80EC0895052E092607FA440FE6
:1011D000551F5F3F79F0AA27A51708F051E0479502
:1011E000880F991F9F3F31F0BB27B91708F091E096
:1011F000879508959F919F911124E3CF97FB880FC6
:10120000991F9F3F31F0BB27B91708F091E08795F0
:1012100008959F919F911124D4CF6627772788271F
:1012200099270895D1DF01D0B4CF992339F0552300
:1012300029F09F575F57950F13F49AF1F1CF91580A
:101240009F3FE1F3629FA12D0F92BB27639FA00DEB
:10125000B11DEE27729FA00DB11DEE1FAF93AA27FF
:10126000649FB00DE11D739FB00DE11DAA1F66279D
:10127000829FB00DE11DA61F5527749FE00DA11D93
:10128000551F839FE00DA11D561F849FA00D511D6A
:10129000852F7A2F6E2F1F900F9088231AF4939525
:1012A00039F48FCF000C111CBB1F661F771F881FDE
:1012B00001280895629FD001739FF001829FE00D85
:1012C000F11D649FE00DF11D929FF00D839FF00DC5
:1012D000749FF00D659FF00D9927729FB00DE11D71
:1012E000F91F639FB00DE11DF91FBD01CF0111244E
:1012F0000895A1E21A2EAA1BBB1BFD010DC0AA1F57
:10130000BB1FEE1FFF1FA217B307E407F50720F06E
:10131000A21BB30BE40BF50B661F771F881F991FE9
:101320001A9469F760957095809590959B01AC0132
:06133000BD01CF0108958C
:061336000425386C640080
:00000001FF
